:10000000405A001081030000890300008B030000A8
:100010008D0300008F030000910300007E90FFEF2E
:10002000000000000000000000000000930300003A
:1000300095030000000000009703000099030000F2
:100040009B030000C10300009B0300009B03000012
:100050009B0300009B0300009B0300009B03000028
:100060009B0300009B0300009B0300009B03000018
:100070009B0300009B0300009B0300009B03000008
:100080009B0300009B0300009B0300009B030000F8
:100090009B0300009B0300009B0300009B030000E8
:1000A000CB1700009B0300009B0300009B03000094
:1000B0009B0300009B0300009B0300009B030000C8
:1000C0009B0300009B0300009B0300009B030000B8
:1000D0009B0300009B0300009B0300009B030000A8
:1000E0009B03000000F002F800F05EF80AA090E820
:1000F000000C82448344AAF10107DA4501D100F0E3
:1001000053F8AFF2090EBAE80F0013F0010F18BF51
:10011000FB1A43F0010318471C3400003C34000074
:100120000A444FF0000C10F8013B13F0070408BF1D
:1001300010F8014B1D1108BF10F8015B641E05D0BB
:1001400010F8016B641E01F8016BF9D113F0080F70
:100150001EBF10F8014BAD1C0C1B09D16D1E58BF02
:1001600001F801CBFAD505E014F8016B01F8016B39
:100170006D1EF9D59142D6D37047000000230024AC
:1001800000250026103A28BF78C1FBD8520728BFA7
:1001900030C148BF0B6070471FB59DE8030002F0F7
:1001A000CDFD1FBD10B510BD02F024FE1146FFF7B6
:1001B000F3FF00F0AFFB02F042FE03B4FFF7F2FFE3
:1001C00003BC02F073FE0000D0F800D0D0F804F0B9
:1001D000024600200B21C30700D0802303EB500010
:1001E00012F8013B491E184409B2C0B20029F2D1ED
:1001F000704770477047704770477047443322110B
:10020000FFB559A60446E1CE8DE8E100022902DAE5
:10021000002004B0F0BD6018002100F8011D6946FF
:10022000B3FBF2F502FB1535B3FBF2F34D5D00F8BD
:10023000015DA042F4D8ECE702460020342A01D048
:100240003F2A06D14A78342A03D18978322900D14D
:100250000120704702004FF0000009D0012A0ED0A3
:10026000022A04D1C978662907D0462905D07047EB
:10027000C9786B2901D04B29F9D101207047C97881
:100280006E29FAD04E29F8D07047F0B50646002006
:10029000044605460346F25CA2F13007092F01D857
:1002A000FDB209E0A2F14107052F02D8373AD5B2D5
:1002B00002E0613A052A05D95B1CDBB205EB0414A8
:1002C000042BE8D30988A14200D10120F0BD10B56C
:1002D00002F0D5FA2848294C006840B102F03DFCF4
:1002E000A0F5C820206002F038FC606010BD02F06C
:1002F00034FC6FF448210844206002F02EFC6FF4B7
:10030000C8210844F1E7F8B51C4D034600242E68C7
:100310007018696887188F4200D9881A00920246BF
:10032000304602F037FB2046F8BD0B460146134825
:1003300010B500680024184401F0B4FF204610BD39
:1003400070B500220D4C134608340AE0E65C855C6B
:100350005B1C7540DBB28554402B00D30023521C3C
:10036000D2B28A42F2D370BD3031323334353637AF
:100370003839414243444546CC0000101401001076
:100380000948804709480047FEE7FEE7FEE7FEE729
:10039000FEE7FEE7FEE7FEE7FEE7FEE70448054965
:1003A000054A064B7047000085190000E500000073
:1003B000400A0010405A0010404A0010404A001005
:1003C00010B54FF040210120086001F0D0FD10BDB4
:1003D0000648022141600021016741611D22C2607F
:1003E000C163012141600020704700000000094006
:1003F00010B591FBF2F491FBF2F302FB1411C0E98A
:10040000003110BDA71B000010B50178427801EB48
:10041000810102EB4101C902A1F5C0318AB2C17864
:100420000479303901EB810104EB41014901A1F567
:10043000C06101F4FC611143C27980796FF02F0330
:10044000303800EB800003EB40001044C0F3440060
:10045000084310BDF0B58DB004463022F949684616
:1004600002F01FFCE079A17A00EB4002C2EBC01061
:1004700001EBC001207A64225043627A102302EB20
:10048000820200EB420008444002742100EB41204C
:100490002179627901EB810103EB4101114480B2C2
:1004A00001F01F010143237800206D4655F82020FC
:1004B0001678B3420DD166785778BE4209D1A67836
:1004C0009278964205D14001203000F4F07001434B
:1004D00003E0401CC0B20C28E8D30DB00846F0BDC4
:1004E000D94910B5486980040CD4D84A906843F6BD
:1004F00098239468241A9C42FBD34869800401D451
:10050000012010BD052001F0CBFA002010BD70B510
:10051000CE4CA668042001F0C3FACD4D03E000BF25
:10052000FFF7DEFF48B1A068801BA842F8D308E0BF
:10053000FFF7D6FF08B1012070BDA068801BA8425C
:10054000F6D3002070BD10B5092001F0A9FAC14909
:100550000120487010BD2DE9F041002506462C46CB
:10056000BD4F0BE040222146BB48FFF7DEFE0020D6
:100570003958001D0D444028FAD34034B442F1D319
:100580002846BDE8F081B5A086B00FC88DE80F0001
:10059000B6A0B74900680490086800264FF6FF022D
:1005A0001040B44A40F4807010430860B249B34F21
:1005B0004FF4C8200E60B3493860B1480860B249B2
:1005C0004012B24D0860F8202870FF206870A870B3
:1005D000AF48B046D0F8109001F044FC9D4CDFF8D5
:1005E000B4A24FF0010B606801280FD14FF4C8206E
:1005F000FFF7B1FFE0B3D4F8042020204346514672
:1006000051F822703B54401C4028F9D36268002006
:100610005AF822102A180B5C401C82F8003460281B
:10062000F8D300F0D1FF012000F0F9FF4FF4E17A98
:100630005546514640F2491001F079FC294640F2F6
:100640009F1001F074FCA04601F040F998F80100F9
:1006500045460028F8D100218FA000F071FD04006C
:10066000F2D08E49087A66287DD046287BD0DCE01F
:10067000FFE784F800B003223B680221104601EB3B
:10068000932740F6FF7E13E0B0EB932F01D3714622
:1006900000E0411CC0F3032C4CEA0118A85405EB00
:1006A000020C09098CF80180801C8CF80210D21C05
:1006B0008742E9D8402240F204416748FFF735FEFF
:1006C00065498878032802D3584681F802B0C0B241
:1006D00004AA5746125C60685AF8203083F8432019
:1006E0005AF8203083F827204B786A4602EB131320
:1006F0005AF820C01B788CF844305AF820C08CF887
:1007000029304B7857F820C003F00F031DF8033051
:100710008CF8453057F820C08CF82E300B7857F8FD
:1007200020C002EB13131B788CF8463057F820C01A
:100730008CF83030097801F00F01515C57F8202017
:1007400082F8471057F8202082F8321057F820001E
:100750004030FFF73DFD616857F8211081F82D000A
:100760003D480C3000E01CE0FFF774FE616857F86C
:100770002120A2F8580057F82120A2F8520057F87B
:100780002110A1F8500034481C30FFF73DFE61688D
:1007900057F82120A2F8560057F82110A1F84E0072
:1007A00034E7487A722801D052283ED1887A6D28E1
:1007B00006D04D2804D0782801D0582835D10126FC
:1007C00036480078662801D046282ED140221101F3
:1007D0002148FFF7AAFD012E03D140211E48FFF753
:1007E000AFFD1D492D484F7A001D091DFFF74DFD36
:1007F000D8B16868A84628B14FF4C820FFF7ABFE0F
:10080000F8B112E038462549FFF716FD50B11248FD
:1008100022498079FFF71EFD20B14FF4C820FFF771
:100820009AFE28B1092001F03BF9FFF78CFE0BE797
:100830000A2001F035F900273D46072001F030F984
:100840003EE056E00033000000800920000009402F
:1008500080841E00C8000010BC0700103031323305
:100860003435363738394142434445464B4E4600CD
:100870000CED00E00000FA0510010010000100106E
:10088000005C0600F8000010FC000010BC01001025
:1008900030330000C00000104634320068080010F9
:1008A000A8050DD1204600F025FC0446A0F5706097
:1008B000FF381ED0032C1CD340F6F870844218D2A7
:1008C000402229464848FFF730FD4035012E03D12C
:1008D00040214548FFF734FD09EB0700402242491B
:1008E00000F0EEFC0720403701F0DAF8002DE7D0E9
:1008F000D6E70B2001F0D4F85446514640F29F1041
:1009000001F015FB214640F2491001F010FB88F878
:1009100001B099E601F036F801F040F9FFF758FD13
:1009200001F084F8002001F0BBF801F045FB2F4EE8
:1009300070692F4D2F4CDFF8C08040034FF0000747
:1009400002D5FFF7CDFD70B3042001F0A9F870695E
:10095000800414D4FFF7DBFD28B3FFF7D8FD10B3F4
:10096000FFF7D5FDF8B1042001F09AF8A0684146E0
:100970007269920403D4A268121A8A42F8D3A0685A
:1009800042F21071A268121A8A42FBD3706B10F007
:10099000004F14D501206860FFF799FC4FF4C82080
:1009A000FFF7D9FD58B100F0BFFC00284FF002005E
:1009B0000AD001F075F86868401C02D00AE06F6048
:1009C000F1E700F0ABFC05E001F06AF86868401C54
:1009D00000D16F60FFF77BFCA0684146A268121A45
:1009E0008A42FBD3FFF7CFFDBC070010008009202F
:1009F000C80000100000094080841E002DE9F84363
:100A000000250E460446FE4FA84634E0B4F5007FAC
:100A100019D2132C0DD0142C0ED0B4F5FF7F0ED0AC
:100A2000A4F58070FF380CD03E2C1CD8F548005D32
:100A300012E097F820000FE0388C000A0CE05520F7
:100A40000AE0AA2008E0B4F5006F08D2EE4820447E
:100A5000A0F5805090F8000E8DF8000005E0EB48FE
:100A6000006801280BD08DF80080E9499DF800004E
:100A7000641C48556D1CB542C8D3BDE8F8830122FB
:100A8000A4F500616846FFF750FCEEE770B5DC4D59
:100A90002C6B402C00D94024E86AE96902198A428B
:100AA00002D90C1A042169702146FFF7A7FF2246DC
:100AB000D749822000F05FFEE86A2044E862286B94
:100AC000011BD348296300F19F008268A2EB040256
:100AD000826005D06978022901D00021017370BDC0
:100AE00003216970F9E7CA4910B59F31C948086008
:100AF0000D22822000F03FFEC1490520487010BD44
:100B000070B50D46C4494A69520302D5496D49057D
:100B100021D4B0F5007F1ED3C04BB94CB0F5006FA7
:100B20001AD29968A269891ABD4A914204D3996878
:100B3000A161002161606161B54A00214032B24B80
:100B400007E044181C44565CA4F58054491C84F802
:100B5000006EA942F5D370BD616921B99968A161A0
:100B600099686161A060A949096829B10129F2D198
:100B7000AC4909780029EED199686269891AAA4AB4
:100B8000914217D29968A16199686161A168401A80
:100B90006168884203D9616A884200D26060062099
:100BA00000F07EFF2A466168BDE8704098484030FA
:100BB000FFF7A9BBBDE870400C2000F071BF10B575
:100BC0008F4CA178E06A4218E1698A4206D9081A76
:100BD000A07005206070022000F088FDA178E06A16
:100BE000FFF78EFFA178E06A0844E062206B421AAA
:100BF0008748226300F19F008368A3EB01018160B5
:100C000002D06178052904D100210173BDE81040AC
:100C100069E710BD2DE9F041794CA178E06A4218EE
:100C2000E1698A4206D9081AA07005206070022086
:100C300000F05CFD764B0021A07803F14005E26AEC
:100C400008E056186F5C9E5DBE4202D00021A16292
:100C500002E0491C8142F4D31118E162216B0A1AA7
:100C60006B49226301F19F018B68A3EB0000886050
:100C700002D06078052808D1A06A20B1002008734E
:100C8000BDE8F0412FE70120F9E7BDE8F0816048B9
:100C900010B58030D0F81110027D09BA21F0FF01A3
:100CA0001143574A4902D162C18A49BA49021163C4
:100CB000806888420DD0822000F018FD022000F0EC
:100CC00015FD534902209F310873FFF70CFF0020E8
:100CD00010BD012010BD70B54D48803002248168E0
:100CE00000F11F0529B1007B000607D4022000F0A7
:100CF000FDFC2C73FFF7F7FE002070BD012070BDD6
:100D000010B543483E4C80308068A178884200D2BC
:100D1000A0703F49A2784031822000F02CFD0320D2
:100D200060703B48A2789F308168891A81600021F9
:100D3000017310BD364810B58030816839B1007B31
:100D4000000601D5822000E0022000F0CFFC3049EF
:100D500000209F310873BDE81040C4E610B5FFF7CE
:100D6000BAFF00281FD02A487021403002220170AB
:100D7000002141708270C1700171417181710A223C
:100D8000C271017241728172C172302202730122FA
:100D900042738173C17301744174194912208870C0
:100DA000BDE81040ACE710BD1CB5FFF794FF00286C
:100DB00069D01E480A220621008883B26846FFF7E0
:100DC0001FFA134800224030802302704370827063
:100DD0000121C1702021017143718271C2714122D0
:100DE0000272542242724F2282724C22C2720173EA
:100DF000417381734622C17302745023437417E018
:100E0000DC000010C0320000BC010010CC0000105B
:100E1000BC070010555342530080092000000940D0
:100E2000A0860100C800001020A1070004040000F3
:100E3000722383746923C3746E230375742343750B
:100E40008175C2756C2202766122427673228276A7
:100E50006822C276017741778177C1779DF80110CA
:100E600080F820109DF8021080F821109DF80310E2
:100E700080F822109DF8041080F82310DC4924200B
:100E80008870FFF73DFF1CBD10B5FFF724FF002859
:100E90000CD0D84803210170002141708170C170CD
:100EA000D34904208870BDE8104029E710BD10B573
:100EB000FFF711FF002810D0CE4800210622017054
:100EC00042708170C170017141718171C171C849F5
:100ED00008208870BDE8104012E710BD10B5FFF77C
:100EE000FAFE002815D0C24AC248116A491E0B0EEC
:100EF00003700B0C43700B0A8370C17000210171E9
:100F0000417102238371C17108209070BDE81040C7
:100F1000F6E610BD10B5FFF7DEFE002819D0B54883
:100F20000021B34B0170417081700822C2701A6AAF
:100F3000140E0471140C4471140A8471C2710222DB
:100F4000027241728272C1720C209870BDE810402A
:100F5000D6E610BD2DE9F041A54DA64C0021A8789C
:100F60004034A44A02E0535C6354491C0346814266
:100F7000F9D31F2B72D120689F4988426ED19D4EB4
:100F800060685F364FF001087060A068B060607BF9
:100F900018B9A07B08B1102802D986F80C8059E056
:100FA000E07B1E28F9D00FDC12282ED005DC48B3D8
:100FB0000328F2D1BDE8F041D0E61528EDD01A287B
:100FC000EBD1BDE8F0415FE702272A2828D010DCEA
:100FD00023281DD025281ED02828DED1FFF757FE54
:100FE000002826D0207B000618D56F70BDE8F041A0
:100FF0004CE52F281ED05528CFD05A28CDD1BDE89A
:10100000F04154E7BDE8F04194E6BDE8F041CBE69D
:10101000BDE8F0417EE7BDE8F0415FE7022016E061
:10102000FFF735FE002804D0207B00060ED485F89B
:1010300001802AE6FFF72BFE0028FAD0207B00066D
:1010400004D485F80180C5F828801EE6822000F0CF
:101050004DFB3773BDE8F04145E5FFE7822000F026
:1010600045FB022000F042FB062068700DE6604858
:1010700010B54178022908D003290ED004290FD0D9
:10108000052901D10021417010BD5A484030C07B74
:101090002828F9D1BDE81040F8E4BDE8104022E569
:1010A000822000F023FBF8E710B55249022000F03F
:1010B00031FB4F498870487858B101280CD0022084
:1010C00000F014FB4B4902205F310873BDE810406B
:1010D00009E5BDE810403DE746484030C07B2A287E
:1010E00004D02F2805D1BDE8104093E5BDE810409D
:1010F00065E510BDFFB50246002002EB4205014642
:101100004FF400666C4603AA6B1844F82130B342D2
:1011100002DD002004B0F0BD384F07EB6307DB07AA
:101120003F78575401D03B095354535C8F0003F070
:101130000F035354BB40491C18440329E4DBE9E77F
:10114000F0B505460020044602462C4B4FF40077CC
:1011500000E0641C2E5D36B102EB040C9C449CF84C
:1011600000C4B445F5D0032C3DD302F5806018448B
:10117000047F457FC67F04EB0524857F2D0405EBA6
:1011800006652C4451EA040529D021B9184949685B
:1011900040318C4223D8174C00216C3455181D4423
:1011A00095F800546554491C0C29F7D3817EC27E02
:1011B00001EB0221027D407D120402EB00600C185D
:1011C0002046FFF797FF40F6F57501E0FFF792FF25
:1011D000C11EA942FAD3A0F57061FF3901D00020E9
:1011E000F0BD2046F0BD2032BA42B3D3F0BD0000BE
:1011F000DC000010FC07001055534243BC010010F6
:1012000030B4514C4F4A0323C4F8B031136843F44F
:10121000803313604D4A30BC104710B572B633248A
:101220004B4B10C307C34B484FF47A710068B0FBB7
:10123000F1F01860191D4648FFF7E2FF62B610BDD5
:10124000434A32231360C2E9010142484FF47A71E4
:101250000068B0FBF1F0D06002F114011046CFE756
:101260003B4A34231360C2E901013A484FF47A71D2
:101270000068B0FBF1F0D06002F114011046BFE746
:1012800010B572B60424344951F82420824212D990
:101290003149783951F82410814207D12146084656
:1012A000FFF7CEFF21460846FFF7DAFF2146084642
:1012B000FFF7C6FF02E0641C1D2CE5D962B610BD25
:1012C0002DE9F041254C236803B92060204D002012
:1012D0002835636803E00F5C1E18401CAF55904230
:1012E000F9D398184FF480766060B04213D120682B
:1012F000FFF7C6FF164D1435286800B1FEE7144904
:10130000324628312068FFF788FF286800B1FEE7E1
:101310000020606020600020BDE8F08110494FF49B
:1013200080400860FEF750BF00214FF480404FF42A
:10133000D02208C890421944FBD309B1002070475D
:101340000120704788C10F4000C00F40F11FFF1FF0
:101350007408001094010010A83300005C01001014
:1013600008ED00E0664800214FF001128180017015
:101370004170C0E90221704761491C31002000F032
:10138000C9B910B55E4C1434A288402A00D9402255
:101390008020216800F0EFF9216801442160A188D4
:1013A000081AA08010BD10B5554C002014342168D7
:1013B00000F0B0F9216801442160A188081AA080DA
:1013C00010BD00221146802000F0D5B94D49002003
:1013D00000F0A0B92DE9F041494C00271C34484DDC
:1013E0002178A4F10806082863D2DFE800F062043F
:1013F000647262628381FFF7BFFF2078C00900F04A
:1014000056F9E088B0802078C0F34111F1BB6178D3
:101410000C294AD2DFE801F00609490B49101A1DD0
:101420001F25314201F0A4FD4DE0002000E0012025
:1014300001F0DEFD50B306E010F01F0F35D1A078AB
:1014400040F080002870BDE8F041BAE701F054FD9B
:1014500039E000202AE010F01F0F26D12848401C58
:101460001AE010F01F0F20D101F00AFE70B1FFF753
:10147000A8FFBDE8F04100F071BA00F01F0001289C
:1014800013D1687810B12079A97800E00DE0884286
:101490000BD21B491031084430601CE000F01F00E3
:1014A000012802D101F094FEC4E7802000F01EF96B
:1014B000B780BDE8F081080608D4B0880028F8D0CD
:1014C000FFF771FFB0880028EFD0F2E7BDE8F041E8
:1014D0007CE7080602D5BDE8F04152E7287801060E
:1014E000E7D500F07F002870BDE8F04100F041B87A
:1014F000802000E00020BDE8F04100F001B90000CC
:10150000680100109C09001001460007C00E090682
:1015100000D5401C7047DD491022C1F80822C1F8EF
:10152000100200BFD1F80002C006FBD57047D74AB1
:101530001023C2F80832C2F8100200BFD2F800022D
:10154000C006FBD5C2F80832C2F81012D2F8000269
:10155000C006FBD57047CD493022C1F80822C1F83A
:10156000100200BFD1F800028006FBD5D1F81402AA
:10157000704730B5C649C74D41EA00442146284668
:10158000FFF7D5FF21462846BDE83040CFE7BF48EA
:101590000021C0F848124021C0F84C120122C0F8C6
:1015A0004822C0F84C1200BFD0F80012C905FBD584
:1015B0004FF0FF31C0F83812C0F83412C0F80812EA
:1015C0000C21C0F80412704730B5B34C1A202060CB
:1015D000221D116830EA0101FBD1B04901234B679C
:1015E0008B67AA4D0023C5F810318A23C1F8F83063
:1015F0002060116830EA0101FBD14FF0E0214FF08B
:101600008070C1F88002A64B202283F80024C1F824
:101610000001FFF7BCFFBDE830400020A9E710B58E
:10162000040001D0012000E000204FF4807141EA65
:1016300000419C48FFF77BFF9B494FF480200CB191
:10164000886310BDC86310BD704710B500B101209C
:101650004FF4807444EA00419448FFF768FF8B48D8
:101660000321C0F8441200BFD0F80012C905FBD511
:10167000C0F8084210BD10B502468078FFF744FF5D
:101680008249D1F84432012484402343C1F84432D2
:10169000C1F848029088C1F84C0200BFD1F800029E
:1016A000C005FBD54FF48070C1F8080210BD70472B
:1016B00000B5FFF729FF7E495DF804EB41EA0040E1
:1016C000891334E700B5FFF71FFF79495DF804EB94
:1016D00041EA004077492AE700B5FFF715FF744952
:1016E0005DF804EB41EA0040891320E700B5FFF7FD
:1016F0000BFF6F495DF804EB41EA00406E4916E7C5
:1017000000B5FFF701FF6A495DF804EB41EA0040CC
:1017100089130CE700F00F02012370B503EB82037D
:101720005A4AC2F8283200BFD2F820321C05FBD535
:10173000C3F309030024DD1C05E000BFD2F81862E2
:1017400041F8046B641CB4EB950FF7D30021C2F889
:10175000281241F24821C140C9070AD1FFF7D4FE3F
:101760004FF4A06141EA0040FFF7D5FE5348FFF770
:10177000D2FE184670BD70B513460546434C00F0C6
:101780000F00022202EB8000C4F82802C4F82432C1
:101790000020DA1C05E000BF51F8046BC4F81C629D
:1017A000401CB0EB920FF7D30020C4F82802284663
:1017B000FFF7AAFE4FF4A06141EA0040FFF7ABFE3D
:1017C0003F48FFF7A8FE184670BD2DE9F0412F4DA8
:1017D000D5F80032C5F80832180721D53148FFF78F
:1017E0009AFE3848FFF7B7FEC10605D5FFF7CFFED2
:1017F000BDE8F04100F0A3B8810705D5BDE8F04190
:1018000000F0010000F095B8010709D5400703D5A5
:10181000BDE8F04100F09AB8BDE8F04100F09DB895
:10182000294E58074FF001071CD4BDE8F081002471
:10183000D5F8302207FA04F10A4210D06008C5F842
:10184000381200BFD5F800128906FBD5D5F814125E
:10185000E2070CD056F8201009B103208847641C19
:10186000202CE5D3D5F830020028E0D1DDE73CB9E3
:10187000490705D5316819B1012088470124D7E708
:1018800056F820100029EAD00220E7E700C008201F
:10189000000180000005D000F4CF082000C0024005
:1018A00018E000E00005FE00008009200005D800D7
:1018B0000005400000012000000101000005F200C9
:1018C0000005FA000002FE00C434000070B5284C88
:1018D000607820B30026274D012810D002280DD1B2
:1018E000A8686168401A2449884215D32348406B90
:1018F000400011D50120FFF792FE667070BDA86808
:101900006168401A1E498842F8D30020FFF787FE1D
:10191000A86860600220607026700C2005E02078C6
:101920000028EBD1012020700D20BDE8704000F0B0
:10193000B7B8002802D10E4901204870704710B591
:10194000FFF710FD0A490020487010BD084801212A
:1019500041700849896841607047704770470228A4
:1019600003D0032803D1FFF782BBFFF79DBB70476D
:101970008C01001000000940A086010000800920B1
:1019800040420F0030B52648244A2021C0F8A0115B
:10199000D0F8A0114906FBD50121C0F80C1109238C
:1019A000C0F88430C0F88010AA23C0F88C305524C9
:1019B000C0F88C40D0F888506D05FBD52325C0F8C1
:1019C000A450C0F8A010C0F8AC30C0F8AC4000BFC4
:1019D000D0F8A8305B05FBD540F20113C0F8043104
:1019E00040F20123C0F80831C0F800110421C0F80A
:1019F000A8110C49C0F8C4100021C0F8C811D0F8D3
:101A0000B03143F00303C0F8B03145F23A0303604C
:101A1000054801600D20106030BD000088C10F40F6
:101A200000C00F40CE9FF8F708ED00E0002070479F
:101A30005849C20702D04FF000728A67800702D56A
:101A40004FF080608867002070475249C20702D07B
:101A50004FF00072CA67800702D54FF08060C867F8
:101A600000207047014600204A4ACB0703D0536F3D
:101A70009B0100D50120890704D5516F490101D58B
:101A800040F00200704710B50446FFF7EBFF034635
:101A9000FFF7DBFF24EA0300FFF7CAFF002010BDB9
:101AA00010B53D4B38B159680424042906D2DFE84B
:101AB00001F0061D375400205860986010BD0428BE
:101AC00007D005280AD0012402285ED001284CD076
:101AD00010BD0320FFF7B9FF01201EE0BDE8104054
:101AE0000120B2E7FFF7A4FF5C6010BD062808D014
:101AF0000328FAD00928ECD00D280AD00C28E8D009
:101B000010BD0320FFF7A1FF0220FFF791FF022085
:101B100021E00320FFF799FF0220BDE8104087E78E
:101B2000062808D00A280FD009281ED00C28D0D0AB
:101B30000D28EED010BD986810F01F0F00F10100C5
:101B40009860F7D102201DE00320FFF77EFF0120FF
:101B5000FFF76EFF0320586010BD07280AD00A283F
:101B6000B7D00B2811D00928F6D10320FFF76DFF5D
:101B70000120B7E7986810F01F0F00F1010098608E
:101B8000EAD10120BDE810407DE70320FFF75DFFAB
:101B90000220A7E700800920A4010010F0B5AB499E
:101BA000032008630020C1F80801A94804228265C7
:101BB000026C42F004020264A64A8A6600220A61AC
:101BC0001022C261026822F0100202600322C1F8F2
:101BD0007022C1F8742200224A644FF400328261FC
:101BE000026842F4003202600922C1F80021C1F803
:101BF00004211022C1F8D42052048263026A42F404
:101C0000001202620D22C1F8D020C1F8E0200022AB
:101C1000C1F8F4204FF00052C263026A42F0005251
:101C200002620022C1F8F0204FF08052C263026AC3
:101C300042F0805202621022CA6702048261026886
:101C400042F0004202601022C1F81421202787656B
:101C5000026C42F0200202641022C1F81C21802292
:101C6000C265026C22F0800202649026C1F8FC601A
:101C70000204C263026A22F0004202621022C1F82A
:101C8000DC20D204C263026A22F400020262012252
:101C90000A66CA654A660323C1F8D8300523C1F82D
:101CA000E4308A601123CB60CA630B640224C1F85C
:101CB00020411225C1F824510C604D600C604D602C
:101CC00010248C659405C461046844F480040460A5
:101CD0000124CC630B641023C1F82C31CB14C365F1
:101CE000036C43F4006303641023C1F830318B1498
:101CF000C365036C43F48053036440F282234B6258
:101D00009A240C62CB6110234B618761036843F016
:101D10002003036010238B6140248461036843F037
:101D20004003036001230B67CB6640F20243CB62A2
:101D30008B621023C1F8E83093068363056A45F08F
:101D4000806505621025C1F8EC50D506C563056AAB
:101D500025F0006505624E635503C561056825F4ED
:101D6000005505600025C1F8E4515506C567056EAC
:101D700045F0007505660025C1F8E851C367036E9C
:101D800043F0806303668A23C1F8F8300823C1F862
:101D9000C8309504C563066A46F48026066210269C
:101DA000C1F828610E15C665066C26F480660664C7
:101DB0000126C1F88060C1F88460C1F89060C1F864
:101DC000A060C1F8A460C1F8A860C1F8BC6000269A
:101DD000C1F81861C465046C44F0400404640B65E8
:101DE0001405C461046824F480140460CB64D40432
:101DF000C461046824F4002404608B64C561046831
:101E000024F4802404600024C1F80C418365036C31
:101E100043F008030364C1F8104110238365036C89
:101E200043F0100303640C480C4B0068984204D143
:101E300041F8B82F8A60CA60F0BD094A9042FBD1D0
:101E4000812041F8B80F8860C860F0BD00C0024032
:101E5000008009200200010064010010473F19279B
:101E6000473F19474D4900200867C86002224A6170
:101E700088613022CA634A498A684A49C1E9002018
:101E80004949086049490860784649490860002086
:101E900070472DE9F04341F288320024424F434E0F
:101EA000434B904208D8642800D228B942F21072FD
:101EB000914201D8052907D28620386078463460DF
:101EC00018608620BDE8F083DFF8D490D9F8085078
:101ED000344AD2F800C0A5EB0C05D2F804C00CEBD4
:101EE0004C08C8EBCC1CB5EBCC0F06D205203860F3
:101EF0007846346018600520E4E7284D4FF0020C66
:101F0000C5F804C048B1DFF8AC80B8FBF0F0401071
:101F1000A861C5F804C001206860D9F80800C2E9CA
:101F200000013C607846346018600020CAE770B554
:101F30001C4C00250E466560FFF7ABFF1A490006F2
:101F400001D5086870BD164B06EB46022068C2EB4F
:101F5000C6129E68361AB6EBC20FFAD30F48022299
:101F60004260C26B02F0FE02C2636560E9E70C48A2
:101F700080680C490A68801A4A6802EB4203C3EB86
:101F8000C212B0EBC20F08D3044802224260C26BF7
:101F900002F0FE02C26300204860704700800040EB
:101FA00000000940B0010010D0000010D400001063
:101FB000D800001080C3C90119480621016107211A
:101FC000016000214161416202214160C168C9068E
:101FD000FCD400E08168C1684907FBD40020704749
:101FE0000F498860C868C006FCD48868704700B58F
:101FF0000B46024604E000BF12F8010BFFF7F0FFAA
:102000005B1EF9D200BD00B50B46024604E000207D
:10201000FFF7E6FF02F8010B5B1EF8D200BD0000DF
:102020000000034070B500BF00BF00BF00BF00BF8D
:1020300000BF00BF00BF00BF00BF00BF00BF00BFA8
:1020400000BF00BF00BF00BF00BF00BF00BF00BF98
:1020500000BF00BF00BF00BF00BF00BF00BF00BF88
:1020600000BF00BF00BF4025CE4CE5610620FFF752
:10207000B7FFA56100BF00BF00BF00BF00BF00BF2A
:1020800000BF00BF00BF00BF00BF00BF00BF00BF58
:1020900000BF00BF00BF00BF00BF00BF00BF00BF48
:1020A00000BF00BF00BF00BF00BF00BF00BF00BF38
:1020B00000BF00BF70BD2DE9FC5FBB4DBB4EBC4FE8
:1020C0005FEA020A8B4604464FF000080DD001A9D2
:1020D000B84800F001F980B18220286021203060EA
:1020E000784638608220BDE8FC9FC5F800807846BD
:1020F000C6F8008038600020F5E703208DF8000066
:10210000200C8DF80100200A8DF802008DF80340A4
:1021100000BF00BF00BF00BF00BF00BF00BF00BFC7
:1021200000BF00BF00BF00BF00BF00BF00BF00BFB7
:1021300000BF00BF00BF00BF00BF00BF00BF00BFA7
:1021400000BF00BF00BF00BF00BF00BF00BF00BF97
:10215000944C4FF04009C4F81C9004216846FFF7E6
:1021600046FF51465846FFF74EFFC4F8189000BF8F
:1021700000BF00BF00BF00BF00BF00BF00BF00BF67
:1021800000BF00BF00BF00BF00BF00BF00BF00BF57
:1021900000BF00BF00BF00BF00BF00BF00BF00BF47
:1021A00000BF00BF00BF00BF00BF00BF00BF9CE773
:1021B0002DE9FC47044601A97E4800F08DF87A4DD0
:1021C0007A4EDFF8EC9148B18220286022207946CF
:1021D00030608220C9F80010BDE8FC879DF804003B
:1021E000800701D4FFF71EFF20208DF80000200992
:1021F0008DF8010020018DF8020000248DF80340C5
:1022000000BF00BF00BF00BF00BF00BF00BF00BFD6
:1022100000BF00BF00BF00BF00BF00BF00BF00BFC6
:1022200000BF00BF00BF00BF00BF00BF00BF00BFB6
:1022300000BF00BF00BF00BF00BF00BF00BF00BFA6
:102240004027DFF86081C8F81C7004216846FFF75A
:10225000CEFEC8F8187000BF00BF00BF00BF00BFAF
:1022600000BF00BF00BF00BF00BF00BF00BF00BF76
:1022700000BF00BF00BF00BF00BF00BF00BF00BF66
:1022800000BF00BF00BF00BF00BF00BF00BF00BF56
:1022900000BF00BF00BF2C60794634600020C9F841
:1022A000001099E770B5414D414E3F4C2AB1FFF700
:1022B00002FF000609D5206870BD86202060092035
:1022C000286078463060862070BD0020206028603D
:1022D00078463060002070BD2DE9F041364C0F4645
:1022E0000646A56806E0A068401BB04202D3012064
:1022F000BDE8F081384600F003F80028F3D1F7E795
:1023000070B5044600BF00BF00BF00BF00BF00BFE4
:1023100000BF00BF00BF00BF00BF00BF00BF00BFC5
:1023200000BF00BF00BF00BF00BF00BF00BF00BFB5
:1023300000BF00BF00BF00BF00BF00BF00BF00BFA5
:1023400000BF00BF4025174EF5610520FFF748FE8E
:102350000020FFF745FE2070B56100BF00BF00BF41
:1023600000BF00BF00BF00BF00BF00BF00BF00BF75
:1023700000BF00BF00BF00BF00BF00BF00BF00BF65
:1023800000BF00BF00BF00BF00BF00BF00BF00BF55
:1023900000BF00BF00BF00BF00BF207800F00100F9
:1023A00070BD000000800920D0000010D400001093
:1023B000D8000010A0860100000009402DE9F34F6D
:1023C00085B0044603A9B24800F0FDF8B14DB24E05
:1023D000B24F4FF0820B18B12120C5F800B060E079
:1023E000FFF720FE42208DF800004FF0000ACDF8E4
:1023F00001A0CDF805A0ADF809A000BF00BF00BF47
:1024000000BF00BF00BF00BF00BF00BF00BF00BFD4
:1024100000BF00BF00BF00BF00BF00BF00BF00BFC4
:1024200000BF00BF00BF00BF00BF00BF00BF00BFB4
:1024300000BF00BF00BF00BF00BFDFF864924FF0D5
:102440004008C9F81C800B216846FFF7D0FDC9F889
:10245000188000BF00BF00BF00BF00BF00BF00BFAB
:1024600000BF00BF00BF00BF00BF00BF00BF00BF74
:1024700000BF00BF00BF00BF00BF00BF00BF00BF64
:1024800000BF00BF00BF00BF00BF00BF00BF00BF54
:1024900000BF03A97E4800F096F848B12220C5F895
:1024A00000B0306078463860822007B0BDE8F08F19
:1024B0009DF80C00800701D4FFF7B4FD02208DF8D1
:1024C0000000200C8DF80100200A8DF8020006980B
:1024D0008DF803408DF8040000BF00BF00BF00BFAF
:1024E00000BF00BF00BF00BF00BF00BF00BF00BFF4
:1024F00000BF00BF00BF00BF00BF00BF00BF00BFE4
:1025000000BF00BF00BF00BF00BF00BF00BF00BFD3
:1025100000BF00BF00BF00BF4446C846C9F81C400A
:1025200005216846FFF763FDC8F8184000BF00BFEB
:1025300000BF00BF00BF00BF00BF00BF00BF00BFA3
:1025400000BF00BF00BF00BF00BF00BF00BF00BF93
:1025500000BF00BF00BF00BF00BF00BF00BF00BF83
:1025600000BF00BF00BF00BF00BF00BFC5F800A094
:102570007846C6F800A03860002096E72DE9F05FA5
:10258000444EDFF81491DFF814A1150083460F467E
:102590004FF000080ED000240AE0395D0BEB040078
:1025A000FFF70CFF000602D53068BDE8F09F641C01
:1025B000AC42F2D3C6F800807946C9F8008000200A
:1025C000CAF80010F1E72DE9F041364C0F460646F7
:1025D000A56806E0A068401BB04202D30120BDE818
:1025E000F081384600F003F80028F3D1F7E770B522
:1025F000044600BF00BF00BF00BF00BF00BF00BF58
:1026000000BF00BF00BF00BF00BF00BF00BF00BFD2
:1026100000BF00BF00BF00BF00BF00BF00BF00BFC2
:1026200000BF00BF00BF00BF00BF00BF00BF00BFB2
:1026300000BF40251A4EF5610520FFF7D1FC0020B0
:10264000FFF7CEFC2070B56100BF00BF00BF00BF28
:1026500000BF00BF00BF00BF00BF00BF00BF00BF82
:1026600000BF00BF00BF00BF00BF00BF00BF00BF72
:1026700000BF00BF00BF00BF00BF00BF00BF00BF62
:1026800000BF00BF00BF00BF207800F0010070BD98
:10269000A0860100D0000010D4000010D800001067
:1026A00000800920000009402DE9F047FE4E8046D9
:1026B0004FF0807730684024FC4DB84249D100BFCC
:1026C00000BF00BF00BF00BF00BF00BF00BF00BF12
:1026D00000BF00BF00BF00BF00BF00BF00BF00BF02
:1026E00000BF00BF00BF00BF00BF00BF00BF00BFF2
:1026F00000BF00BF00BF00BF00BF00BF00BFEC6154
:102700001520FFF76DFC0020FFF76AFC00F0FF09C1
:10271000AC6100BF00BF00BF00BF00BF00BF00BF73
:1027200000BF00BF00BF00BF00BF00BF00BF00BFB1
:1027300000BF00BF00BF00BF00BF00BF00BF00BFA1
:1027400000BF00BF00BF00BF00BF00BF00BF00BF91
:1027500000BF00BF00BF00BF00BF00BF00BF00BF81
:1027600000BF00BF00BF00BF00BF00BF00BF00BF71
:1027700000BF00BF00BF00BF00BF00BF00BF00BF61
:1027800000BF00BF00BF00BF00BF00BF00BF00BF51
:1027900000BFEC610620FFF723FCAC6100BF00BF67
:1027A00000BF00BF00BF00BF00BF00BF00BF00BF31
:1027B00000BF00BF00BF00BF00BF00BF00BF00BF21
:1027C00000BF00BF00BF00BF00BF00BF00BF00BF11
:1027D00000BF00BF00BF00BF00BF00BF00BF00BF01
:1027E00000BF00BF00BF00BF00BF00BF00BF00BFF1
:1027F00000BF00BF00BF00BF00BF00BF00BF00BFE1
:1028000000BF00BF00BF00BF00BF00BF00BF00BFD0
:1028100000BF00BF00BF00BF00BF00BFEC610120D0
:10282000FFF7DEFB4FEA8800FFF7DAFB3068B842BB
:1028300002D14846FFF7D4FBAC6100BF00BF00BF28
:1028400000BF00BF00BF00BF00BF00BF00BF00BF90
:1028500000BF00BF00BF00BF00BF00BF00BF00BF80
:1028600000BF00BF00BF00BF00BF00BF00BF00BF70
:1028700000BF00BF00BF00BF00BFBDE8F0872DE96B
:10288000F0474FF0000900BF00BF00BF00BF00BF0E
:1028900000BF00BF00BF00BF00BF00BF00BF00BF40
:1028A00000BF00BF00BF00BF00BF00BF00BF00BF30
:1028B00000BF00BF00BF00BF00BF00BF00BF00BF20
:1028C00000BF00BF00BF4025784EF5619F20FFF795
:1028D00087FB0020FFF784FB00F0FF080020FFF7D4
:1028E0007FFBC4B20020FFF77BFBC1B2B56100BF24
:1028F00000BF00BF00BF00BF00BF00BF00BF00BFE0
:1029000000BF00BF00BF00BF00BF00BF00BF00BFCF
:1029100000BF00BF00BF00BF00BF00BF00BF00BFBF
:1029200000BF00BF00BF00BF00BF00BF00BF604DC1
:10293000604E614FB8F1C20F01D1202C07D0822028
:1029400028602120306078463860822095E756481C
:10295000142912D0152913D0162915D0182916D0EC
:10296000C0F800900020FFF79FFEC5F80090784661
:10297000C6F80090386000207FE74FF4801101E036
:102980004FF400110160EDE74FF48001FAE74FF0DA
:102990008071F7E72DE9FF4F8DB00D46DDF86890A7
:1029A0000026434C07935FEA09013ED04FF480575D
:1029B00001463A466846FDF71BFDDDE900B10C9182
:1029C0003A46691C6846FDF713FDDDE90010CDE9C4
:1029D00004013A4668460F99FDF70AFDDDE90085D6
:1029E000A9EB0607C5F58050B84200D2074625B1CD
:1029F000D8457DD10C9885427AD14FF4805000F0B3
:102A0000B5F85FEA000A1CD0D8455BD10C98854226
:102A100058D12A464FEA08305146FFF74CFB0006D2
:102A200019D5504600F0D1F885E086202060214875
:102A300009210160784620490860862011B0BDE870
:102A4000F08F822020601B482221016079461A48BD
:102A500001608220F2E70598804509D1049901EBD5
:102A60000030C1F580525144FFF725FB0006D8D451
:102A70004046FFF79DFB0006D3D407983A468119DC
:102A800005EB0A0000F0C8F8EA194FEA0830514691
:102A9000FFF774FD0006C4D4059988453ED104981B
:102AA00000EB0130049909E0B80100100080092012
:102AB000D0000010D4000010D8000010C1F58052E2
:102AC000514427E0059988450AD1049800EB01306C
:102AD0000499C1F580525146FFF7EDFA0006A0D4E3
:102AE0004046FFF765FB00069BD40798811900E07C
:102AF00018E00F983A463044FFF740FD000690D4A6
:102B0000059988450AD1049800EB01300499C1F574
:102B100080525146FFF732FD000682D4504600F045
:102B200054F80AE007983A4681190F983044FFF7A5
:102B300025FD000601D5206880E73E44002508F108
:102B400001084E45FFF44CAF0549002020600860A5
:102B5000784604490860002070E703480068704721
:102B6000D4000010D8000010B801001070B506465F
:102B700000F0CAF8056806F10B0020F00704B44223
:102B80009CBF002070BD2B466A68BAB11068A04295
:102B900010D304F1080188423CBF5068586007D345
:102BA0005168101941601168091B01605860146078
:102BB000101D70BD13465268002AE7D121462846F1
:102BC00000F0A8F80028DED170BD70B50446051FDE
:102BD00000F09AF80068002C14BF446870BD002C07
:102BE00018BFAC423CBF20466468F8D301680A189D
:102BF000AA4218BF456003D12A6805461144016006
:102C000028684119A1421CBF6C6070BD6168696091
:102C100021680844286070BD032A40F2308010F01B
:102C2000030C00F0158011F8013BBCF1020F624467
:102C300098BF11F801CB00F8013B38BF11F8013BF8
:102C4000A2F1040298BF00F801CB38BF00F8013BA5
:102C500011F0030300F02580083AC0F0088051F815
:102C6000043B083A51F804CBA0E80810F5E7121D20
:102C70005CBF51F8043B40F8043BAFF30080D2073F
:102C800024BF11F8013B11F801CB48BF11F8012B0B
:102C900024BF00F8013B00F801CB48BF00F8012B2E
:102CA000704710B5203AC0F00B80B1E81850203AB8
:102CB000A0E81850B1E81850A0E81850BFF4F5AFDC
:102CC0005FEA027C24BFB1E81850A0E8185044BF66
:102CD00018C918C0BDE810405FEA827C24BF51F8D3
:102CE000043B40F8043B08BF7047D20728BF31F8C7
:102CF000023B48BF11F8012B28BF20F8023B48BF18
:102D000000F8012B7047000000487047E4090010EC
:102D10007047704738B504460A4600206946AFF34D
:102D20000080002808BF38BD02460099204600F008
:102D30003FF8012038BD012000F054B8F8B5AFF3DA
:102D40000080054600200C46102000BF0646A8194A
:102D5000A0420DD9324669460020AFF3008007003B
:102D600008BF00F03FF80098A04218BF0546C419FC
:102D7000FFF7CAFF05600746F01D20F0070046195F
:102D8000284600F00AF8B44208BFF8BDA21B31463D
:102D90003868BDE8F84000F00BB800210160C0E9D8
:102DA000011070471020704700487047DC09001080
:102DB000034640688C46002818BF88423CBF034643
:102DC0004068F8D318681844884207D00CF1030013
:102DD00020F00700001D411A521A0146081D0A6022
:102DE000FFF7F3BE10B500F039F8BDE8104000F071
:102DF0002FB870477546FFF7D7FFAE460500694606
:102E0000534620F00700854618B020B5FDF7C6FAF6
:102E1000BDE820404FF000064FF000074FF00008DB
:102E20004FF0000B21F00701AC46ACE8C009ACE85C
:102E3000C009ACE8C009ACE8C0098D46704710B5C0
:102E40000446AFF300802046BDE81040FDF7B5B959
:102E5000002801D000F02AB87047000010B5012802
:102E600005D0002103A000F027F8012010BD09A122
:102E7000F8E7000053494752544D454D3A204F75ED
:102E800074206F662068656170206D656D6F727962
:102E9000000000003A2048656170206D656D6F721A
:102EA0007920636F7272757074656400014918202F
:102EB000ABBEFEE72600020070B505460C460A20B0
:102EC00000E06D1C00F011F835B128780028F8D129
:102ED00002E0641C00F009F814B120780028F8D151
:102EE000BDE870400A20AFF3008008B569468DF850
:102EF00000000320ABBE08BD194810B5007810F0E3
:102F00001F0F1748C07829D115490839012806D064
:102F1000134A0228937806D003281FD112E01148E3
:102F20000860122012E01048002204E004780CB17E
:102F300044882044521C9342F8D1027872B1086050
:102F4000408803E009481844086000788A88824273
:102F500000D98880FEF715FA012010BD002010BDB1
:102F6000840100102034000032340000533400008B
:102F700070B51D481C4D0078A5F1080510F01F0420
:102F80000AD01948A5F11401184B4A780079012C90
:102F900006D0022C26D109E01348183828601DE01D
:102FA00002B3897888421DD2002015E000F08F041A
:102FB000200605D504F00F064FF48030B04001E044
:102FC0000120A0400AB922070CD18A68024209D028
:102FD000C9680142E8D0012018802B60FEF7D1F9C2
:102FE000012070BD002070BD840100109C090010FC
:102FF00070B502462148A0F11C04017811F01F03AE
:103000000146498804D0012B29D0022B27D111E099
:10301000012924D132B10120FEF716FBA08840F02F
:10302000020005E00020FEF70FFBA08820F0020060
:10303000A08021E0007900F08F00030605D500F0A4
:103040000F034FF480359D4001E0012585406378F2
:103050002BB1030703D0A3682B4200D009B1002095
:1030600070BD22B1FEF742FBE068284303E0FEF7A3
:1030700047FBE068A843E060012070BD84010010B8
:103080002DE9F84F504F00200090B8784FF000091C
:103090004FF0010A4FF4803BA7F11C0600286AD0CC
:1030A0004A4C64E06078022804D0042840D0052807
:1030B0005BD140E06179B878814237D17070207976
:1030C000B070414900200C3901F80090401C0428E0
:1030D000FAD301254FEA06080AFA05F0D8F80810D5
:1030E000084202D02846FEF7EDFAD8F808100BFA8D
:1030F00005F0084203D045F08000FEF7E3FA6D1CAE
:10310000102DE9D34FF00110C8E902090120FEF7A4
:103110009CFAE0794006B8F8040002D540F00100BE
:1031200001E020F00100A8F804001EE060881DE026
:10313000E078009019E00098B8B9A07800F08F0509
:10314000280604D505F00F010BFA01F001E00AFA98
:1031500005F0B16801432046B160FEF78CFA2846BD
:10316000FEF7A6FA2846FEF7B7FA2078044420783E
:10317000002897D11FE086F8019001245546D846D3
:10318000B16805FA04F0084202D02046FEF79AFA28
:10319000B16808FA04F0084203D044F08000FEF75A
:1031A00091FA641C102CEBD34FF00110C6E9020910
:1031B0000020FEF74AFAB8787178884202D10120DF
:1031C000BDE8F88F0020FBE78401001032340000D6
:1031D0002DE9FC5F384D00273E466878BB46B8466F
:1031E000002866D0BA46354C05F11C095DE06078D0
:1031F000022804D0042808D0052854D119E06079A9
:10320000697888424FD060884EE0A77899F804101A
:10321000E6784FF00008B94245D199F80200B04273
:1032200041D125484FF0010A103010F807B0C655BB
:1032300039E099F80410B94235D1A17801F08F0135
:103240000191090605D5019901F00F024FF4803173
:1032500001E0019A01219140009199F80200B042E9
:1032600013D1A8680843A860E96800988143204604
:10327000E960FEF700FA0198FEF71AFA0198FEF7E6
:103280002BFA009948EA01080DE05E450BD118EAD7
:10329000010F08D1A8688843A860E8688843E860FF
:1032A0000198FEF70FFA20780444207800289ED178
:1032B0005046BDE8FC9F0000680100103234000059
:1032C000EB3C904D53444F53352E30000202010029
:1032D0000110000004F802000100010000000000DD
:1032E00000000000000029EFBEADDE41544F4C202D
:1032F000465072696E7446415431322020200000DD
:10330000143500000435000020350000243500008D
:103310003035000018350000103500000C35000075
:103320001C350000283500002C3500000835000051
:10333000000000000010000000200000003000002D
:10334000004000000050000000600000007000001D
:10335000008000000090000000A0000000B000000D
:1033600000C0000000D0000000E0000000F00000FD
:103370000000010000800100000002000080020047
:10338000000003000080030000000400008004002F
:103390000000050000800500000006000080060017
:1033A0000000070000800700FF0F0000FF1F000063
:1033B000FF2F0000FF3F0000FF4F0000FF5F0000F5
:1033C000FF6F0000FF7F0000FF8F0000FF9F0000E5
:1033D000FFAF0000FFBF0000FFCF0000FFDF0000D5
:1033E000FFEF0000FFFF0000FF7F0100FFFF010073
:1033F000FF7F0200FFFF0200FF7F0300FFFF0300CB
:10340000FF7F0400FFFF0400FF7F0500FFFF0500B2
:10341000FF7F0600FFFF0600FF7F0700FFFF07009A
:10342000120110010000004051C2031300010420EA
:103430004801090220000101008032090400000255
:10344000080650620705820240000007050202409C
:10345000000000040309041C03410054004F004C09
:10346000002000200020002000200020002000205C
:10347000002000280346005000720069006E0074AE
:1034800000200046006C00610073006800200020EE
:1034900000200020002000200020001A03460069C0
:1034A0000072006D0077006100720065003000302E
:1034B00000300030000E034D0065006D006F00729B
:1034C00000790000D5130000000000005F19000023
:1034D00000000000000000000000000000000000EC
:1034E00000000000000000000000000000000000DC
:1034F00000000000000000000000000000000000CC
:103500000000000046656200446563004175670085
:103510004A756C004A616E004A756E005365700012
:103520004D617200417072004F6374004E6F7600FF
:103530004D6179005435000000000010BC0100000E
:1035400020010000FC350000BC0100108458000080
:103550007C010000A00D41544F4C20465072696E12
:1035600074280546D4284B3D39609F4574616C6FC3
:103570006E609920126612341232124E1230120FFF
:103580001BDE30071230122E12663272326D1E466A
:1035900034324E30011546524D202008BC41973739
:1035A000383738263D6E2B38024340061B10600426
:1035B000411AFF01014C100D455F5553494E475FBD
:1035C0004D4F5645B81328085838365F54554E4568
:1035D0005F4550494C4F47551F8A291F175348498B
:1035E00046543103392A0810080E270780C3C90141
:1035F000148793031B6CDCE90116000030C80A6FC6
:103600007C9017481B88B436277C40B68EFE275C1A
:10361000AB8B180AB2203D66C140A3C1AD3AACBF26
:10362000B4292636CA2A3973645FC26D88C57B1DEA
:1036300075C441901596F0FBF5F8E202C817BA5F21
:1036400072CFBDF09F5C1C3187667D0EE6C2297D7E
:10365000EB7E14F7C983515EE7CBD32F8A5F4ABB59
:10366000400055C4FB844942CB790A422F54FB44A5
:10367000EA92CAB77A1B9872520D5436D153B7C921
:1036800024ECF3D27B5C38CDC3537FC2AF89FC7F7F
:1036900008E6A628425EBF772C56076A31540F39D8
:1036A000DB07005AB494967A45B9F859FF032F29DD
:1036B000D52CCF6F432087C4F1FC4348E83E0E6110
:1036C00089147AFE2DD12D02DC490B9DEFC93BBB3D
:1036D000DBA2BA5EC67ECADC872F032B3A313C914F
:1036E0008CD7815C9580879392A02BD8190008FD18
:1036F0006375ABF50010306D2AA5856937C5693251
:10370000C6C52B8BC70AAD66FD0F594C660A93E3FD
:103710007F71EF4A80E28A0035DEDE84663359F23B
:1037200093EB5E774DA7BA9A360EF9C1F655AFFA0C
:1037300095356E1CEF943C503D2F0932CC22F1960A
:10374000E7C7271E31FB465CD7E027BE6F082F3640
:103750003826589C48DC9B2E33B29F13C59E7C159F
:10376000D3E78ACA7397FF85EF1CED411C9B05A91F
:10377000DC7331588576FABE0CCA29FBBC9575A25C
:103780002B04DE5637DCC973BA3FE6552C5238C1DC
:1037900077B7A23E0D4F0C782933423B91BB1D4BAE
:1037A000EC23E586CFCBE4F2F50E44E492EE9BD811
:1037B0000BFD5DF2198DBB50456F1B2C40AF884D42
:1037C0005EF69BC01AB67D7665905EE42D210E8074
:1037D00023BC0EE8962A3C25FE862F79AC7EEBBCF6
:1037E000CD5F14B8B625CCE77F7AD4EEEBC8717EF6
:1037F0000C779FC6B08106E1E9A9966E1930971142
:1038000041FBD293E4CFB457BA0EDE155217772C92
:103810005C167966F1E509B11738DE93C883103676
:103820009F2A907690CDFB50F934B58D6D7B436B1C
:103830003F020E36CEB8A0DC6FDDD8FAECDB8CA1EF
:103840009239199F5D6731DA0E6BD87CD68C30E8DF
:10385000C028E99C371F36A940406C385C15DEF65D
:103860002A5CF7253282BD4C0D9BC9E4217F6D6D2A
:10387000C6F7A99E50BB92CA5C66F2E8AAB6FEE102
:1038800042906BEBBCD4009785E41DB863E371C133
:10389000DA7317014BA4FD93C597B87F51FEDCE99D
:1038A0005A70AEEDB672EA3600FB34D9D704B9A42B
:1038B000B303EEE963720D9BDC7FCDFF89A2471C49
:1038C0007370F8B8FE33F3B4C43D5F118792A97AE0
:1038D00083F33D6E9F5F67A21C46EC7CEE3F113A7E
:1038E0005660D24F09D136AF84B9C75BA9B25A57D7
:1038F0002346E77476EDE5B9E89D0BFA7A0201AA52
:10390000D75D2BC0AD17E80FC948712113A00B2359
:10391000E9624EA89A78B80483C343E87C54CB6527
:103920000AE46AA6A72A62601B3FFBAC06CC0441EE
:1039300091C725EDA8D47108F162ED02D77BB79449
:10394000FB0ABA4BA88052061469F7D6FBD155235F
:1039500089D030E05EAB0D51647B5579B2BD39251D
:10396000DFB1AE722E168FDF47B2FF79554B650877
:1039700073F0A8923FD7504EC486B811C8BFEE7EF0
:10398000C0DADF1BE7584571803A05A85CC98ED3C1
:103990007BCE9D7F0BC96F805579125CC8EF13E811
:1039A000BEC09271C5B63BD28FCEA0A36EF839D3FC
:1039B00059460A7EFFBFCDCA246A5B5520EBE968F1
:1039C0005CE199CA8E1D37AB806593CEE8DDEE7E53
:1039D0008905BF74587541ADC12BC9F767CD19462C
:1039E00093552F8D7267A09871FA1E8C2A92512DD3
:1039F000BEE627935F99B840E6EA66E195AB636D52
:103A000085319AEF61A672C54529E865CFC1565147
:103A1000330F0DE76E2BF1FD9341709664B1FCBE40
:103A2000693C3745111157A6370C07853EAF3F4E0D
:103A300053D54917B51CD973B165E6307ACD4041ED
:103A400027C2EA0DBF1D4BA1E312B5977A7B0EDBAF
:103A50008F807A8E47EFF0C5C234117C701B911DA8
:103A6000BFF4A4DA242345FA512E9785DC6C5CD38D
:103A70004071659C220E09565C91B9257C206BE64D
:103A80009CE58B2C503F5974FFC53B60B73E459178
:103A9000D8BBB4C1EB86BE475001798A2A203EE4E8
:103AA00060AE614884455FED576438104F7C68A470
:103AB0006A8309FD2F943B47E06AB683F8D152D759
:103AC000B8007CC4E308355453B31709007A8784DF
:103AD000BD0F7D6822A282CB773671322DC631D3DD
:103AE0007BC00DC995461DF651271CCA4A569568DC
:103AF000FAA3614A46A02D2A0F9CD93F82A8259A95
:103B000084AAB581BC90085F52DD809FB689F60219
:103B1000DFC9D74E8027690A84E3583E892D181DD6
:103B20009D0C43D71525FCA70979A0B5A57284F68D
:103B3000F660458FA584D528088052BB473EB41D4A
:103B4000A19BF28FDD14A8ECF093859E63AEC0D1EB
:103B5000807E6DCCD61F4B302A213D184F9A8E5255
:103B6000E47ECCB21A3584E3C621FAE8ABA865003E
:103B7000A2A1CE4B64B7B482DC3B8396A3CEE1E72F
:103B8000DA9540410794E24D4C702BFEAD6D5B8C95
:103B9000221B667A48A9624E410155AC116F22A2E0
:103BA00021CA7B91073196A87582C9CFDBAFFCAAE9
:103BB000798B47813383005F237A06BB2AE4CCD616
:103BC0004B333EC7897DDA2843F5F123908E6C6430
:103BD000D3438D18657BA4A9405D5B77626A47AFCC
:103BE000124131DA379C5EDEE0BE78510D9B0D83C9
:103BF00008DE48EC8A5A60EFA47155DBB61BAAE8D0
:103C00001BD8E8952129D0E423C8AD5AEB3EB8E192
:103C1000BF08F75FF0D7A92C2C8E216BB827D0F600
:103C2000B14001B46C5913F18EF9CA9F2CE6F64DE0
:103C30001FD774CCD04F5926C148605F8A9FDC21C2
:103C4000FDBE9BAD194AC2C67BE3C2F77275E96837
:103C5000BB93DE746507C3B19D533A7731C4AE5749
:103C600048729381987C9054DD26DB71C30CB8A315
:103C7000A162DDB8EFA42C86F1CFFB68E6294837B6
:103C8000EF4F28F8CC232625814EE46E71D5F27AC9
:103C9000FD49707E7FF7501D37B6D927FA11C0262F
:103CA000B446AF5C228EF72204E90079C710C6E45F
:103CB000417FB705CDEE21E6D22CBCDF4E65AF17B4
:103CC00014A00CEFB33A9A54DC2514E411E97A13EA
:103CD000A0498125057B3FAEA44E700C01B9B0030D
:103CE000D836ECB141D8FF626B14473CB5F8ACDB79
:103CF0001F397968E0ECEBEDD7AC2E4990BCABB244
:103D000069D51058932866ED9EF314C0010D75FF18
:103D10001254DBB768E7750E82A6A111769D1C8F41
:103D20008C49BFA45B1E68FA2F58B29389DF52A654
:103D3000F0C869C4CF0FCA3D6FD34BD8033782F2A6
:103D4000ADAC3BDF75879600E994414D22B7342630
:103D5000CC572E118389DDDC84C8FF25FE9EE298B6
:103D6000EE18CAD775334AF22BD07D83E3CECC2927
:103D700083605F5897138E63938C1C6700E99A8663
:103D8000D320A64C530A36EA5C5D7C5484C2D5BD70
:103D9000E1204F09CBEE2B56427BEAFD678B40D4E6
:103DA000E41809599D1C1CBF3D10D0E51FF766C2E1
:103DB0005DF38642762185E5F38C878048C8C4236D
:103DC00098EB7B22CA771EC525EEFD47B03DBAA70A
:103DD000FB9E3AF3855971CDAA68C41DDE3414AD3B
:103DE0002D8506DCD74E1E1A932111CEDCCF991FEC
:103DF000D322C929F80A1C932EFBF085798DA47A69
:103E000047129C69C0009340522B2DCF6CE489C1AE
:103E1000F33876ACE7006BCD6E769EB231D35DE0C1
:103E2000046BF308684DDC8DC6CE413136F47D86D7
:103E3000A5958BC3E1F1CC4C7ED611B5615842906B
:103E40004C6E3706CC91C7432819AAF444682F401A
:103E50003FA722CD6FCFA9410403855C08D8EFE8C6
:103E6000FB2825C17ED7ECB8A3662C18591943034B
:103E70009AEAAC316F206BE54EB369667FA1C2E46C
:103E8000D61571DEAC89234EC689D195B3C7EFA391
:103E9000BC225F7DF2609814722B727772CBC704DC
:103EA000DCF67D4B6050D586227592C58ABEEECE7B
:103EB00097C0A1748D18AAF434A05925AB6A0EF5E9
:103EC000390764DAF71A1522D67D4C9B66D1C525D1
:103ED0009B1822208CB040354E2624F58D8FD5EAD4
:103EE00039080B70CA667104B4733F21DD7ECBC9FB
:103EF000ED6974282999BD8DF4258B14C351612077
:103F0000E46A22ECEBE9C101F7CF601B47325B8822
:103F100082D2BFBF161D8F225D7E0FCE7544F73D46
:103F200099DDC97D4B12FDBB0C7415D982FB18E1DC
:103F30008E842E64AA51702171BEC75B4C4FECC6B3
:103F4000EC18D3930502ECDBCA8B45916DBE48900B
:103F5000168B17929C512EDDF642C624E04935F8A7
:103F600019E97D6A5134F79AB8C56C068210A25CD3
:103F7000DC6CF973F15DA4F0B40279A24C40278E99
:103F800032B293058CC0F625E2C07CB5E5A5389B1E
:103F90009916B1BA5DAAF5AFB0CCF0070C1C05ECD0
:103FA00084E391218081862293C75440FC1E5AB835
:103FB000E028AF1B66C9CF65340BFF3EFAB8C2C11B
:103FC000B2A6CE726126B7A874E629F94541FE74FF
:103FD000E81DFE0E6A63D4C37C692C80E1A6262806
:103FE000DB70C355245BE6D2B277B2A04763B0540E
:103FF000268EC153F6458A4E995F8AC6688F5C90BB
:00000001FF
